:04FFF00023001E00CC
:08FFF800000000000000000001
:03000000022FE0EC
:0C2FE00078FFE4F6D8FD75817F023027F1
:1036D20057502053657175656E63657200302E39DF
:0D36E200004175672031392032303036004C
:02340A008F260B
:10340C00E4F527F528C3E5289526E52794005023F5
:10341C00900000AF82AE83E4FCFD7B107A27F9F8B4
:10342C00D31213304003A380EA0528E52870D60593
:03343C002780D214
:01343F00226A
:103524007BFF7A3679D212375E1237F17F76123802
:10353400117BFF7A3679DF12375E1237F17BFF7A1F
:093544003679E312375E0237F11B
:102D60001237961237D4123720E4F524E4F5257D86
:102D700001AF251235747F0112340AE4FDAF25122C
:102D800035740525E525C3940340E40524E524C3F3
:102D9000940540D812380E7B017A01799C75360073
:102DA00075370CE4FFFE12338690019CE064AB7033
:102DB00004A3E064CD60391237FF90019C74ABF03E
:102DC000A374CDF0A37401F0E4A3F0A3F0A3121355
:102DD000BD3D4CCCCDE49001A5F0A304F0E4A3F0FC
:102DE0007B017A01799CF53675370CFFFE1233C8EA
:102DF00090019EE0D39405400374C0F0C39001A0FD
:102E0000E0943C90019FE094004006E4F0A3743B02
:102E1000F020970B7D017F011230ECD2AF80FE9045
:102E2000019EE0FDE4FF1230ECD2AF123524E4F550
:102E30000E12364FD20EA296920BA297920C12331C
:102E40003EE50E60FCE4F50E12147912373680F17F
:03380E00C21622BD
:1035E400AD07AC062016FDD216EC5401F5F1EDF54D
:1035F400F330AF0320EF0AE5F130E7FBC216AFF278
:04360400227F0022FF
:0434CE00AB07AA0698
:1034D2002016FDD216EA5401F5F1A2AF9200C2AF56
:1034E2008DF2EBF5F3A20092AF30AF0320EF07E5C8
:0634F200F130E7FBC216F9
:0134F80022B1
:04347400AB07AA06F2
:103478002016FDD216EA54014420F5F1A2AF9215A8
:10348800C2AF8DF2EBF5F3A21592AF30AF0320EF88
:0834980007E5F130E7FBC21665
:0134A0002209
:10359A002016FDD21675F131A2AF9200C2AF8FF29A
:1035AA00E4F5F3A20092AF30AF0320EF07E5F13064
:0435BA00E7FBC21653
:0135BE0022EA
:0537FA00E4FD0234743F
:0537FF00E4FF02359A11
:0300730002000385
:0600030053F17FC216322A
:0A3386008E318F328B338A34893583
:10339000E4F538F539C3E5399537E53895365027E2
:1033A000E5322539FFE5313538FE1235E4AB33AA75
:1033B00034A935853982853883EF1211C40539E582
:0733C0003970D2053880CE00
:0133C70022E3
:0A33C8008E318F328B338A34893541
:1033D200E4F538F539C3E5399537E53895365027A0
:1033E200E5322539FFE5313538FEAB33AA34A9354C
:1033F200853982853883121185FD1234CE0539E56F
:073402003970D2053880CEBD
:0134090022A0
:1031DF00256C660025303264253032642E2530345C
:1031EF00642C25630025303364253032642E25305E
:1031FF0034642C256300252E33660025332E31666B
:10320F0000244750524D422C412C302E30302C4C44
:10321F002C253033642C253033642C002C002C30BB
:10322F0030302E302C00573A002C523A002C423AB4
:01323F00008E
:043804004101270057
:0A362C00E0FF7E007B017A0079AB1D
:10363600EF7803C333CE33CED8F92420FFE43EFE21
:0936460075360075370802338661
:1036EF00EF7803C333CE33CED8F92420FFE43EFE68
:0936FF007536007537080233C866
:103240002094028028900126E004F0E0FF90019F86
:10325000E0FCA3E0FDD39FEC940050359001A6E084
:10326000601E24FE60248000900126EDF078AB7C87
:10327000007D017B017A0179287E007F08021146DA
:1032800090019FA3E0900126F022E4900126F080B7
:083290000390012612362C22E6
:10306C00E4F531F532E53225E02458F8E4F608F6BB
:10307C000532E532700205316414453170E7E4F530
:10308C0031F53212116CFF600CB42009740129F96E
:10309C00E43AFA80EEEF6043AE02AF010532E5325E
:1030AC00700205311425E02458F8A60608A607126C
:1030BC00116CFF600D642C6009740129F9E43AFA73
:1030CC0080EDEF600CE41211B20429F9E43AFA80B5
:0F30DC00028008E5326414453170A8AE31AF327E
:0130EB0022C2
:1025B500753AFF753B31753CDF753D01753E01751B
:1025C5003F481222E4E4FBFA79C87842900148E0DA
:1025D500FCA3E0FDA3E0FEA3E0FF120CAD120E0686
:1025E500900150EEF0A3EFF0900148E0FCA3E0FD70
:1025F500A3E0FEA3E0FFC004C005C006C00790012C
:1026050050E0FCA3E0FDE4120DCDE4FBFA79C878B7
:1026150042120BA4A804A905AA06AB07D007D00649
:10262500D005D004120AAF9001481213B1900148A9
:10263500E0FCA3E0FDA3E0FEA3E0FF120E0690017F
:1026450052EEF0A3EFF0900148E0FCA3E0FDA3E01B
:10265500FEA3E0FFC004C005C006C007900152E01C
:10266500FCA3E0FDE4120DCDA804A905AA06AB075D
:10267500D007D006D005D004120AAF900148121336
:10268500B1900148E0FCA3E0FDA3E0FEA3E0FFE478
:10269500FBFA79707842120BA49001481213B1909D
:1026A5000152E0FCA3E0FDE4120DCDE4FBFA7970E4
:1026B5007842120CADC004C005C006C00790015099
:1026C500E0FCA3E0FDE4120DCDD003D002D001D093
:1026D50000120AB3C004C005C006C007E4FBFA79BE
:1026E500617845900148E0FCA3E0FDA3E0FEA3E08E
:1026F500FF120CADD003D002D001D000120AB39066
:10270500014C1213B1AB34AA35A93612116CFF6412
:10271500576004EFB4531790014CE0FCA3E0FDA310
:10272500E0FEA3E0FF120DB790014C1213B190012A
:0C2735004CE0FCA3E0FDA3E0FEA3E0FFED
:012741002275
:10360800753AFF753B31753CDF753D01753E0175B7
:103618003F371222E4900137E0FCA3E0FDA3E0FE6F
:03362800A3E0FF1D
:01362B00227C
:082B20008F348E338D328C31AD
:102B28001237C7120E06900148EEF0A3EFF0AF344B
:102B3800AE33AD32AC311237C7C004C005C006C0D1
:102B480007900148E0FCA3E0FDE4120DCDA804A91C
:102B580005AA06AB07D007D006D005D004120AAFE5
:102B6800E4FBFA79707842120BA490014E1213B16B
:102B780090014EE0FCA3E0FDA3E0FEA3E0FF120EEF
:102B88000690014AEEF0A3EFF090014EE0FCA3E0BE
:102B9800FDA3E0FEA3E0FFC004C005C006C0079087
:102BA800014AE0FCA3E0FDE4120DCDA804A905AAA2
:102BB80006AB07D007D006D005D004120AAF9001A3
:102BC8004E1213B17F007E407D1C7C4690014EE082
:102BD800F8A3E0F9A3E0FAA3E0FB120BA4120E0697
:102BE80090014CEEF0A3EFF07538FF753931753A66
:102BF800E3900148E0FEA3E08E3BF53CA3E0FEA392
:102C0800E08E3DF53EA3E0FEA3E08E3FF540E4FFF5
:102C1800FEFDFCAB34AA33A932A831120D4A500488
:102C28007F5380027F4E8F417B017A0079BC121A54
:072C38008D7B017A0079BCDD
:012C3F002272
:082C40008F348E338D328C318C
:102C48001237C7120E06900148EEF0A3EFF0AF342A
:102C5800AE33AD32AC311237C7C004C005C006C0B0
:102C680007900148E0FCA3E0FDE4120DCDA804A9FB
:102C780005AA06AB07D007D006D005D004120AAFC4
:102C8800E4FBFA79707842120BA490014E1213B14A
:102C980090014EE0FCA3E0FDA3E0FEA3E0FF120ECE
:102CA8000690014AEEF0A3EFF090014EE0FCA3E09D
:102CB800FDA3E0FEA3E0FFC004C005C006C0079066
:102CC800014AE0FCA3E0FDE4120DCDA804A905AA81
:102CD80006AB07D007D006D005D004120AAF900182
:102CE8004E1213B17F007E407D1C7C4690014EE061
:102CF800F8A3E0F9A3E0FAA3E0FB120BA4120E0676
:102D080090014CEEF0A3EFF07538FF753931753A44
:102D1800F4900148E0FEA3E08E3BF53CA3E0FEA35F
:102D2800E08E3DF53EA3E0FEA3E08E3FF540E4FFD4
:102D3800FEFDFCAB34AA33A932A831120D4A500467
:102D48007F5780027F458F417B017A0079BC121A38
:072D58008D7B017A0079BCBC
:012D5F002251
:1034F9007538FF753932753A05E4FBFA797A7844FB
:10350900120CAD8F3E8E3D8D3C8C3B7B017A007950
:0B351900BC121A8D7B017A0079BC22E5
:103672007538FF753932753A0A8F3E8E3D8D3C8C16
:103682003B7B017A0079BC121A8D7B017A0079BCEE
:013692002215
:10333E00C210E49000B7F0900126F012362CE4FF94
:10334E00FE7D207C419001A1E0F8A3E0F9A3E0FA14
:10335E00A3E0FB120BA49000B81213B1E490011C71
:10336E00F0C211A294B3920FA297B3920CD2A0F511
:08337E0057900125F002002622
:10147900A20C309701B3500AA297920C209703123D
:101489003240900125E0600B14F0E07006FD7F0208
:10149900123574E5576005D55702D2A01237B8EF57
:1014A9007003021A301236B48F269001A7E0600348
:1014B900200E05AF26123811E52624F8603324FEE4
:1014C900604C24E6600C240360030219F7C20E0283
:1014D90019EFE4900127F0E0FF04F074CC2FF582B6
:1014E900E43400F583E526F07D017F02123574802E
:1014F900AB900127E0D394004003E014F07F081279
:10150900354D7F2012354D7F0812354D808E900163
:1015190027E024CCF582E43400F583E4F0200E0EB4
:10152900D20E7B017A0079CC121EA00219EF7B0141
:101539007A0079CE900134EBF0A3EAF0A3E9F01236
:1015490013579001301213B17F437E4D7D527C5069
:10155900900130E0F8A3E0F9A3E0FAA3E0FBC3129D
:10156900134660030219EF7B017A0079CC12306CC3
:10157900855D82855C83E0644160030219E2AA5EAD
:10158900A95FC0038B34856035856136D003122588
:10159900B59000A31213B1AA62A9637B01C0038BA2
:1015A90034856435856536D0031225B59000A712B8
:1015B90013B1AA68A9697B01123608900121121397
:1015C900B12010499000B7E004F0E0C3940A500339
:1015D9000219EFD2109000A3E0FCA3E0FDA3E0FE06
:1015E900A3E0FF9001281213B19000A7E0FCA3E04B
:1015F900FDA3E0FEA3E0FF90012C1213B17D017F52
:101609000212357490012574C8F00219EF9000A7F1
:10161900E0FCA3E0FDA3E0FEA3E0F5358E348D33B5
:101629008C32A3E0FCA3E0FDA3E0FEA3E0F5398E34
:10163900388D378C36A3E0FCA3E0FDA3E0FEA3E0E0
:10164900F53D8E3C8D3B8C3A753E01753F007540EA
:10165900B375410175420175431D9000A3E0FCA3D8
:10166900E0FDA3E0FEA3E0FF120076900126E0FF73
:10167900D394004006EF14F52D80028F2D7538FFA5
:10168900753932753A10753B00852D3C900126E07D
:10169900753D00F53E7B017A0079CC121A8D9000D8
:1016A900ABE0FCA3E0FDA3E0FEA3E0FF122B208B3F
:1016B900318A3289337B017A0079CC1232987531BB
:1016C900FF75323275332B7B017A0079CC1232984F
:1016D9009000AFE0FCA3E0FDA3E0FEA3E0FF122C25
:1016E900408B318A3289337B017A0079CC12329866
:1016F9007531FF75323275332B7B017A0079CC1243
:1017090032989000B3E0FCA3E0FDA3E0FEA3E0FF64
:101719001234F98B318A3289337B017A0079CC1200
:1017290032987531FF75323275332B7B017A007926
:10173900CC12329890011DE0FCA3E0FDA3E0FEA3CA
:10174900E0FF1236728B318A3289337B017A007954
:10175900CC1232987531FF75323275332D7B017A8F
:101769000079CC123298A20F309401B3500620941C
:1017790003123240A294920F752756E4F52890017E
:10178900A5E07046E4FFFE7D7A7C449001A1E0F873
:10179900A3E0F9A3E0FAA3E0FB120BA49000B3E0E5
:1017A900F8A3E0F9A3E0FAA3E0FB120D4A40030213
:1017B900188F7D017F021235749001257464F0C27F
:1017C900A075274112324002188F201103021860B8
:1017D9009000B8E0FCA3E0FDA3E0FEA3E0FF9000C9
:1017E900B3E0F8A3E0F9A3E0FAA3E0FB120D4A6025
:1017F9000A400890011CE004F08005E490011CF007
:1018090090011CE0D3940340387D017F02123574A6
:101819009001257464F0752741123240E4FFFE7D82
:10182900207C419001A1E0F8A3E0F9A3E0FAA3E04C
:10183900FB120BA49000B81213B1C211E490011C61
:10184900F09000B3E0FCA3E0FDA3E0FEA3E0FF906D
:1018590000B81213B1802FE4FFFE7D7A7C44900119
:10186900A1E0F8A3E0F9A3E0FAA3E0FB120BA4902E
:1018790000B3E0F8A3E0F9A3E0FAA3E0FB120D4AF4
:101889005004D211C2A07531007532007533277B1F
:10189900017A0079CC123298E4F52CF52A752B01DE
:1018A9007B017A0079CC12000EC3E52B9FEE648090
:1018B900F8E52A648098501974CC252BF5827400B8
:1018C900352AF583E0622C052BE52B70D3052A8098
:1018D900CF9001A7E070157B017A0079CC12375EB1
:1018E9007F2A123811AF2C12370880647BFF7A32B5
:1018F900793512375EE52D04FF1237087F2C12382F
:1019090011900126E004FF1237087BFF7A327938FB
:1019190012375E9000B3E0FCA3E0FDA3E0FEA3E074
:10192900FF120E067B007A0079001228B07BFF7A3D
:1019390032793C12375E90011DE0FCA3E0FDA3E083
:10194900FEA3E0FF120E067B007A0079001228B090
:101959001237F1900121E0F8A3E0F9A3E0FAA3E03E
:10196900FB90011DE0FCA3E0FDA3E0FEA3E0FF1254
:101979000AAF120E068E2A8F2BD3E52B94B4E52AD3
:1019890064809480400C7498252BF52B74FE352ABD
:10199900F52AC3E52B944CE52A6480947F500C7496
:1019A90068252BF52B7401352AF52AC3E52B9405F7
:1019B900E52A6480948050047D01801FD3E52B942F
:1019C90005E52A648094804004E4FD80027D017F5E
:1019D900011235747D01E48009E4FD7F011235743B
:1019E900E4FDFF123574E4900127F00214A590017B
:1019F90027E0FF04F074CC2FF582E43400F583E589
:101A090026F0900127E0B40A0C900125E07006FD4C
:101A19007F02123574900127E0C3945050030214D9
:071A2900A5E014F00214A572
:011A30002293
:10379600E4F5847585FF53912FF592F5A475A5FF81
:0137A6002200
:10372000C214E4FDFF123574E4FD7F01123574E428
:06373000FD7F020235746A
:10357400EF1460101460162402701ABD0103C2A770
:1035840022D2A722BD0103C2A622D2A622BD0103D4
:06359400D28022C2802259
:10378400EF24FD700CD214750DFA7D017F02123501
:0237940074229D
:10373600E50DD39400400CD50D09C214E4FD7F02BB
:0437460012357422A2
:1034400025640020200053657474696E67733A0028
:1034500041727269766552616E67653D00206D004C
:103460005365714D6F64653D004379636C654D6FC5
:0434700064653D0052
:061EA0008B2E8A2F893011
:101EA6001235BFAB2EAA2FA93012116C900137F054
:101EB60012141720E0411EEE422077432194441E5F
:101EC600EB451FB84C208F4E225C50212C511EE74B
:101ED6005221C2532191561F2257215759000022E1
:101EE6006543A208220237FFAB2EE5302402F9E44F
:101EF600352FFA753AFF753B34753C40753D0175D3
:101F06003E01753F461222E4900146A3E090019EF1
:101F1600F0D39405400374C0F00220D0AB2EE53018
:101F26002402F9E4352FFA12306CAA58A9597B011C
:101F3600C003753AFF753B34753C408B3D753E01D9
:101F4600753F46D0031222E4AA5AA95B7B01C0035F
:101F56008B34855C35855D36D0031225B590013C02
:101F66001213B1AA5EA95F7B01C0038B348560356D
:101F7600856136D0031225B59001401213B1900148
:101F860046E0FEA3E0FFD39400EE64809480500305
:101F9600022265D3EF943CEE6480948040030222D3
:101FA60065EF24FFFFEE34FFFE7B017A01793C02E8
:101FB60036EFE4900144F0A3F090019FE0FEA3E029
:101FC600FF900144E0FCA3E0FDC39FEC9E400302AA
:101FD6002265C3ED943CEC64809480400302226544
:101FE600900144E0FEA3E0FF7B017A01793C1236C2
:101FF60036900145E02401FF900144E03400FE33B1
:1020060095E0FDFC7B007A0079001228B07BFF7A10
:1020160034794312375E90013CE0FCA3E0FDA3E077
:10202600FEA3E0FF122B20900139EBF0A3EAF0A308
:10203600E9F012375E7BFF7A34794312375E9001FE
:1020460040E0FCA3E0FDA3E0FEA3E0FF122C4090DD
:102056000139EBF0A3EAF0A3E9F012375E1237F18B
:10206600900145E004F07006900144E004F0021F80
:10207600BF1237FFE490019FF0A3F07B017A01794C
:102086009CF53675370C0221BDAB2EE5302402F9DE
:10209600E4352FFA753AFF753B34753C40753D01C2
:1020A600753E01753F461222E4900146E0FEA3E02C
:1020B600FF90019FEEF0A3EFF0C3943CEE94004036
:1020C6000990019FE4F0A3743BF07B017A01799CAF
:1020D60075360075370CE40221BDAB2EE5302402BF
:1020E600F9E4352FFA753AFF753B34753C40753D7A
:1020F60001753E01753F461222E4900146E0FCA3BD
:10210600E0FDEC120DCDE4FBFA797A7844120CADC1
:102116009001A11213B17B017A01799C7536007585
:10212600370CE40221BDAB2EAA2FA9309000021273
:102136001185B444089001A57401F08005E490016E
:10214600A5F07B017A01799C75360075370CE48021
:1021560066AB2EAA2FA93090000212118524CF60FB
:102166000E24DF601180009001A67401F0800DE45A
:102176009001A6F080069001A67402F07B017A0118
:10218600799C75360075370CE4802C023524AB2E0D
:10219600AA2FA930900002121185B431089001A728
:1021A6007401F08005E49001A7F07B017A01799C27
:1021B60075360075370CE4FFFE0233C87BFF7A34B0
:1021C600794612375E1237F17BFF7A34795012372F
:1021D6005EE4FFFE7D7A7C449001A1E0F8A3E0F97D
:1021E600A3E0FAA3E0FB120BA4120E067B007A0012
:1021F60079001228B07BFF7A34795D12375E123788
:10220600F17BFF7A34796012375E9001A5E07004A5
:102216007F4180027F441238111237F17BFF7A34F6
:10222600796912375E9001A6E0600F24FE60130400
:1022360070169001387448F0800E9001387431F0B1
:1022460080069001387452F0900138E0FF12381180
:0F2256001237F10237F17D017F011230EC80FE6B
:012265002256
:10002600E4F529F528F527F526AB29AA28A927A856
:1000360026AF29AE28AD27AC26120AAFC004C005EC
:10004600C006C007AB29AA28A927A826AF29AE282B
:10005600AD27AC26120AAFD003D002D001D00012D1
:0A0066000CAD8F0B8E0A8D098C087B
:01007000226D
:080076008F318E308D2F8C2E8E
:10007E009001371213BD3B5CA8F190013B1213BDEA
:10008E004AC2A72890013F1213BD29612E13900179
:10009E00431213BD42652EE0900137E0F8A3E0F95C
:1000AE00A3E0FAA3E0FBE4FFFE7D807C3F120AAFE3
:1000BE009001471213B1900143E0F8A3E0F9A3E0D9
:1000CE00FAA3E0FBAF31AE30AD2FAC2E120CAD1259
:1000DE0027D2900147E0F8A3E0F9A3E0FAA3E0FBF2
:1000EE00120BA490014B1213B1900143E0F8A3E060
:1000FE00F9A3E0FAA3E0FBAF39AE38AD37AC361258
:10010E000CAD1227D2900147E0F8A3E0F9A3E0FA74
:10011E00A3E0FB120BA490014F1213B190014BE020
:10012E00FCA3E0FDA3E0FEA3E0FFA804A905AA0638
:10013E00FB120BA4E4FBFA7980783F120AB3122F5C
:10014E003AA804A905AA06AB07E4FFFE7D807C3F12
:10015E00120CAD9001531213B190014BE0FCA3E0D1
:10016E00FDA3E0FEA3E0FF900153E0F8A3E0F9A3A6
:10017E00E0FAA3E0FB120BA49001571213B1900109
:10018E004FE0FCA3E0FDA3E0FEA3E0FFA804A90559
:10019E00AA06FB120BA4E4FBFA7980783F120AB38D
:1001AE00122F3AA804A905AA06AB07E4FFFE7D802C
:1001BE007C3F120CAD90015B1213B190015BE0FC21
:1001CE00A3E0FDA3E0FEA3E0FF900153E0F8A3E05F
:1001DE00F9A3E0FAA3E0FB120BA490015F1213B196
:1001EE0090014FE0FCA3E0FDA3E0FEA3E0FF900131
:1001FE005FE0F8A3E0F9A3E0FAA3E0FB120BA490F2
:10020E0001631213B190014BE0FCA3E0FDA3E0FEED
:10021E00A3E0FF900163E0F8A3E0F9A3E0FAA3E006
:10022E00FB120BA49001671213B1AB35AA34A9339C
:10023E00A832AF3DAE3CAD3BAC3A120AAF90014393
:10024E00E0F8A3E0F9A3E0FAA3E0FB120CAD9001F5
:10025E006B1213B190019B740AF090016BE0FCA33A
:10026E00E0FDA3E0FEA3E0FF1227A090017312139E
:10027E00B190016BE0FCA3E0FDA3E0FEA3E0FF1252
:10028E00278A9001771213B1900173E0FCA3E0FD71
:10029E00A3E0FEA3E0FF90015BE0F8A3E0F9A3E08A
:1002AE00FAA3E0FB120BA490014B1213B190015B69
:1002BE00E0FCA3E0FDA3E0FEA3E0FF900157E0F811
:1002CE00A3E0F9A3E0FAA3E0FB120BA4900177E000
:1002DE00F8A3E0F9A3E0FAA3E0FB120BA4A804A98B
:1002EE0005AA06AB07900163E0FCA3E0FDA3E0FEC8
:1002FE00A3E0FF120AAF90014F1213B190014FE02D
:10030E00FCA3E0FDA3E0FEA3E0FFA804A905AA0656
:10031E00FB120BA4C004C005C006C00790014BE041
:10032E00FCA3E0FDA3E0FEA3E0FFA804A905AA0636
:10033E00FB120BA4D003D002D001D000120AB312CC
:10034E002F3A90017B1213B1900177E0FCA3E0FDF0
:10035E00A3E0FEA3E0FF90015FE0F8A3E0F9A3E0C5
:10036E00FAA3E0FB120BA4900167E0F8A3E0F9A357
:10037E00E0FAA3E0FB120AB390017F1213B19001D1
:10038E007FE0FCA3E0FDA3E0FEA3E0F54B8E4A8DDB
:10039E00498C4890017BE0FCA3E0FDA3E0FEA3E0C6
:1003AE00FF12316C9001931213B1900173E0FCA314
:1003BE00E0FDA3E0FEA3E0FF90015FE0F8A3E0F90B
:1003CE00A3E0FAA3E0FB120BA490017BE0F8A3E0FC
:1003DE00F9A3E0FAA3E0FB120CAD9001971213B152
:1003EE00900197E0FCA3E0FDA3E0FEA3E0FF120D59
:1003FE00B7900197E0F8A3E0F9A3E0FAA3E0FB12AF
:10040E000BA4E4FBFA7980783F120AB390018712AD
:10041E0013B1900167E0FCA3E0FDA3E0FEA3E0FFB3
:10042E00A804A905AA06FB120AB39001831213B100
:10043E00E4FFFEFDFC900187E0F8A3E0F9A3E0FAEB
:10044E00A3E0FB120D4A603B4039900183E0FCA310
:10045E00E0FDA3E0FEA3E0FF120DB7900187E0F8E8
:10046E00A3E0F9A3E0FAA3E0FB120CAD90017FE04C
:10047E00F8A3E0F9A3E0FAA3E0FB120AB39001831C
:10048E001213B1900183E0FCA3E0FDA3E0FEA3E014
:10049E00FFA804A905AA06FB120BA4E4FBFAF9783F
:1004AE0040120BA4E4FBFA798078BF120AB39001D4
:1004BE008F1213B1E4FFFE7D407CC0900187E0F8FF
:1004CE00A3E0F9A3E0FAA3E0FB120BA4E4FBFA7994
:1004DE00807840120AB3900137E0F8A3E0F9A3E068
:1004EE00FAA3E0FB120BA4E4FBFA79807840120A1F
:1004FE00B3900187E0F8A3E0F9A3E0FAA3E0FB12C2
:10050E000BA4900137E0F8A3E0F9A3E0FAA3E0FB17
:10051E00120BA4E4FBFA79807841120CAD90018B9A
:10052E001213B190016BE0FCA3E0FDA3E0FEA3E08B
:10053E00FFA31213B190017FE0FCA3E0FDA3E0FE48
:10054E00A3E0FF90018FE0F8A3E0F9A3E0FAA3E0A7
:10055E00FB120BA490018BE0F8A3E0F9A3E0FAA341
:10056E00E0FB120BA4900183E0F8A3E0F9A3E0FAFC
:10057E00A3E0FB120AB390017BE0F8A3E0F9A3E03D
:10058E00FAA3E0FB120BA490018BE0F8A3E0F9A311
:10059E00E0FAA3E0FB120BA4900193E0F8A3E0F9BC
:1005AE00A3E0FAA3E0FB120AB3900197E0F8A3E0F0
:1005BE00F9A3E0FAA3E0FB120BA490016B1213B1A6
:1005CE0090018BE0F8A3E0F9A3E0FAA3E0FBE4FFCF
:1005DE00FE7D807C3F120AAF90016BE0F8A3E0F93C
:1005EE00A3E0FAA3E0FB120BA4900137E0F8A3E01E
:1005FE00F9A3E0FAA3E0FB120BA4C004C005C006E9
:10060E00C007AB35AA34A933A832AF3DAE3CAD3BE3
:10061E00AC3A120AAF900143E0F8A3E0F9A3E0FA76
:10062E00A3E0FB120CADD003D002D001D000120A11
:10063E00B390016B1213B190019BE014F090016B1B
:10064E00E0F8A3E0F9A3E0FAA3E0FBA3E0FCA3E04B
:10065E00FDA3E0FEA3E0FF120AAF1237C790013FE1
:10066E00E0F8A3E0F9A3E0FAA3E0FB120D4A50096B
:10067E0090019BE0600302026890014FE0FCA3E052
:10068E00FDA3E0FEA3E0F54B8E4A8D498C48900108
:10069E004BE0FCA3E0FDA3E0FEA3E0FF12316C9063
:1006AE0001671213B1900173E0FCA3E0FDA3E0FE1D
:1006BE00A3E0FF900153E0F8A3E0F9A3E0FAA3E072
:1006CE00FB120BA4C004C005C006C00790015BE07E
:1006DE00FCA3E0FDA3E0FEA3E0FF900157E0F8A32A
:1006EE00E0F9A3E0FAA3E0FB120BA4C004C005C01E
:1006FE0006C007900177E0FCA3E0FDA3E0FEA3E0B7
:10070E00FF900163E0F8A3E0F9A3E0FAA3E0FB1287
:10071E000BA4D003D002D001D000120AAF8F4B8EA3
:10072E004A8D498C48D007D006D005D00412316CC2
:10073E007BDB7A0F79497840120AB390016312136A
:10074E00B1900147E0F8A3E0F9A3E0FAA3E0FBE4DF
:10075E00FFFE7D807C3F120CAD900147E0F8A3E0D8
:10076E00F9A3E0FAA3E0FB120CADE4FBFA79807872
:10077E00BF120AB3900187E0F8A3E0F9A3E0FAA351
:10078E00E0FB120BA4E4FBFA7980783F120AB31255
:10079E002F3AE4FBFA7980783F120AB390016B127C
:1007AE0013B1E4FFFEFD7CC090016BE0F8A3E0F90D
:1007BE00A3E0FAA3E0FB120AB390016BE0F8A3E00A
:1007CE00F9A3E0FAA3E0FB120CAD90016B1213B18A
:1007DE0090016BE0F8A3E0F9A3E0FAA3E0FBE4FFDD
:1007EE00FE7D807C3F120AAF90018B1213B19001F7
:1007FE006BE0FCA3E0FDA3E0FEA3E0FF90016BE045
:10080E00F8A3E0F9A3E0FAA3E0FB120BA4E4FBFAD1
:10081E0079807840120CADE4FBFA7980783F120AA9
:10082E00B390018BE0F8A3E0F9A3E0FAA3E0FB128A
:10083E000CAD90018B1213B1E4FFFE7DC07C3E9097
:10084E00016BE0F8A3E0F9A3E0FAA3E0FB120BA41E
:10085E0090016BE0F8A3E0F9A3E0FAA3E0FB120B22
:10086E00A4E4FBFA798078BF120AB390016BE0F82A
:10087E00A3E0F9A3E0FAA3E0FB120BA490016F1220
:10088E0013B190017FE0FCA3E0FDA3E0FEA3E0FF27
:10089E0090018FE0F8A3E0F9A3E0FAA3E0FB120BBE
:1008AE00A490016B1213B190018FE0FCA3E0FDA3A5
:1008BE00E0FEA3E0FF90018FE0F8A3E0F9A3E0FAD9
:1008CE00A3E0FB120BA4A804A905AA06AB07E4FF3C
:1008DE00FE7D807C3F120AAF90015F1213B1900132
:1008EE007BE0FCA3E0FDA3E0FEA3E0FFA804A905C6
:1008FE00AA06FB120BA4E4FBFA79807840120BA433
:10090E00E4FBFA794078C0120AB390015FE0F8A3D5
:10091E00E0F9A3E0FAA3E0FB120BA4900183E0F848
:10092E00A3E0F9A3E0FAA3E0FB120BA490016FE0A1
:10093E00F8A3E0F9A3E0FAA3E0FB120BA4E4FBFAA0
:10094E0079C07840120CAD90016BE0F8A3E0F9A3EA
:10095E00E0FAA3E0FB120AAF90016FE0F8A3E0F912
:10096E00A3E0FAA3E0FB120BA4E4FBFA7980784033
:10097E00120CAD900183E0F8A3E0F9A3E0FAA3E036
:10098E00FB120AB390017BE0F8A3E0F9A3E0FAA30F
:10099E00E0FB120BA490016FE0F8A3E0F9A3E0FADC
:1009AE00A3E0FB120BA4900193E0F8A3E0F9A3E0FF
:1009BE00FAA3E0FB120AB390018BE0F8A3E0F9A3CF
:1009CE00E0FAA3E0FB120BA490013BE0F8A3E0F9E0
:1009DE00A3E0FAA3E0FB120BA4900147E0F8A3E01A
:1009EE00F9A3E0FAA3E0FB120BA490015F1213B17E
:1009FE0090015FE0FCA3E0FDA3E0FEA3E0FFAB3EB1
:100A0E00AA3FA940121377900143E0FCA3E0FDA397
:100A1E00E0FEA3E0FF900167E0F8A3E0F9A3E0FA9F
:100A2E00A3E0FB120BA4AB41AA42A943121377AB6E
:100A3E0041AA42A943121357E4FBFA79B478431240
:100A4E000D4A5022AB41AA42A943C003C002C001C5
:100A5E00121357E4FBFA79B47843120AAFD001D0DF
:100A6E0002D003121377AB41AA42A943121357E4E3
:100A7E00FBFAF9F8120D4A60244022AB41AA42A9B2
:100A8E0043C003C002C001121357E4FBFA79B478D5
:0D0A9E0043120AB3D001D002D00312137727
:010AAB002228
:0A37D400E4F5955396BF53A27F223F
:10364F005389F0438901538FFE758C70E4F58A53CB
:10365F00B8FD53B7FDD2A9D28C53890F438990532C
:03366F008FEF22B8
:03000B000237E8D1
:0937E800050E758C70758A003223
:10374A000D0A003031323334353637383941424385
:04375A00444546009C
:1030EC005387BF75985053877FE4F5BABF010543EA
:1030FC00A240800353A2BFE4F5BDED14601514602B
:10310C001A14601F1460242404702575BEF075BF5A
:10311C000B802375BEF075BF05801B75BEF075BFA7
:10312C0002801375BE7075BF01800B75BEB0800335
:10313C0075BE30E4F5BF75BD035391FE4392014358
:10314C0091025392FDC21753B8EF53B7EF43B81027
:10315C00E49000A1F09000A0F09000A2F0D2AC227C
:030023000232F0B6
:1032F000C0E0C083C082C0D075D01030983090003C
:10330000A1E0C3949F50259000A0E0FF04F074005A
:103310002FF582E43400F583E599F09000A1E004F4
:10332000F09000A0E0C394A04002E4F0C29830996D
:0E33300004C299C217D0D0D082D083D0E03230
:103693007D207C4E7E0180027E00A217E4335E60B3
:1036A3000BED1D70011CED4C70EA80ECD2178F9965
:0136B30022F4
:1034A1009000A1E0D394004021A3E0FF04F0740058
:1034B1002FF582E43400F583E0FF9000A1E014F0E1
:0C34C100A3E0C394A04005E4F0227F00CB
:0134CD0022DC
:03381100023693E9
:1036B4007F207E4E9000A1E07010D3EF9400EE9432
:0D36C400004007EF1F70ED1E80EA1234A1D8
:0136D10022D6
:10375E0012116CFF600C123811740129F9E43AFA57
:03376E0080EE22C8
:0F37B8009000A1E0D3940040037F01227F002204
:10370800AB07EB54F0C4540F90374D93FF123811A8
:08371800EB540F93FF0238117E
:0937F1007BFF7A37794A02375E4A
:1035BF0012116CFF601EC3648094E1400ED3EF6460
:1035CF008094FA5006EF24E01211B2740129F9E445
:0435DF003AFA80DC58
:0135E30022C5
:0E28B0008F348E338D328C318B358A368937DA
:1028BE00E4F542EC4D4E4F701EE94A4B70057F30E9
:1028CE00023811AB35AA36A937AF4205428F827551
:1028DE00830074300229F4AE33AD32AC31EC335098
:1028EE0036E5374536453570077F2D123811801481
:1028FE00AB35AA36A937AF4205428F827583007475
:10290E002D1211C4AF34AE33AD32AC311213228F4F
:10291E00348E338D328C31754101753B00753ACA58
:10292E0075399A75383BE4FFFEFDFCAB3BAA3AA91C
:10293E0039A838D312134650030229DFAF34AE3311
:10294E00AD32AC31A8381212908F3F8E3E8D3D8C39
:10295E003CEC4D4E4F7004E541702CE53F2430F5B4
:10296E0040E537453645357007AF401238118014B3
:10297E00AB35AA36A937AF4205428F82758300E583
:10298E00401211C4E4F541AF3BAE3AAD39AC38ABB1
:10299E003FAA3EA93DA83C121205AA06A905A80405
:1029AE00C3E5349FF534E5339AF533E53299F532C4
:1029BE00E53198F531AF3BAE3AAD39AC38E47B0A30
:1029CE00FAF9F81212908F3B8E3A8D398C38022913
:1029DE0034E536453745356010AB35AA36A937850F
:0929EE004282758300E41211C459
:0129F70022BD
:100AAC00020E72E86480F8E933E83360110460F0F8
:100ABC00ED33EC337009E8FCE9FDEAFEEBFF2204B0
:100ACC0060DED3EB9FEA9EE99DE8C2E78CF0C2F7AB
:100ADC0095F0400CE8CCF8E9CDF9EACEFAEBCFFB77
:100AEC00120E3D85D0F05804700320D5B3E8047085
:100AFC00075002B2D5020E7C92D5EC0460F7E4CC20
:100B0C00C0E0C398F8603B94186008400DD0E0FB3F
:100B1C00020E54E4FBFAC9FC8028E830E406E4C970
:100B2C00FBE4CAFCE830E305E4C9CACBFCE8540793
:100B3C006010F8C3E913F9EA13FAEB13FBEC13FC9E
:100B4C00D8F130F52FC3E49CFCEF9BFFEE9AFEED41
:100B5C0099FDD0E0FBEF4E4D4C701222DB03020EE0
:100B6C0079EC2CFCEF33FFEE33FEED33FDED30E78B
:100B7C00EB020E54EF2BFFEE3AFEED39FDD0E0FB0D
:100B8C0050130BBB0003020E7CED13FDEE13FEEFB6
:080B9C0013FFEC13FC020E54E0
:100BA400EC4D6011E8497017ED33EC3304600DE44B
:100BB400FCFFFEFD22E933E8330470F8020E7212E2
:100BC4000E3D58046009E4CC2481500628500902E3
:100BD4000E7C284003020E79C0E0EB4A7044B980D1
:100BE40006D0E0FB020E68EF4E701CBD8008EBFFE0
:100BF400EAFEE9FD80EBE98DF0A4FEE5F0020C8D40
:100C0400E9CDF9EAFEEBFFEF89F0A4FCE5F0CE892B
:100C1400F0A42EFFE435F0CD89F0A42DFEE435F0E8
:100C24008067EF4E7005BD80D780C3EF8BF0A4AC16
:100C3400F0EE8BF0A42CFCE435F0F8EF8AF0A42C51
:100C4400E5F038FCE433CB8DF0A42CFCE5F03BF864
:100C5400EE8AF0A42CFCE5F038F8E433CF89F0A454
:100C64002CFCE5F038CF3400CE89F0A42FFFE5F05A
:100C74003EFEE433C98DF0A42EFEE5F039CD8AF0B2
:100C8400A42FFFE5F03EFEE43DFD33D0E0FB50072A
:100C94000BBB000F020E7CEC2CFCEF33FFEE33FE9B
:060CA400ED33FD020E54C9
:100CAA00020E7CEC5D046005E859047003020E72C2
:100CBA00120E3D580460F6EC4860F2EC7004FDFE3A
:100CCA00FF22C860DB2481C85009C398600250061D
:100CDA00020E799850CAF582E9294B4A7005AB820F
:100CEA00020E6875F0007C1A7880C3EF9BEE9AEDCD
:100CFA0099400DC3EF9BFFEE9AFEED99FDE842F095
:100D0A00DC23ACF0D0E0FFD0E0FED0E0FDAB8220E7
:100D1A00E7101BEB60BAEC2CFCEF33FFEE33FEED71
:100D2A0033FD020E54E803F830E705C0F075F00011
:100D3A00EF2FFFEE33FEED33FD40B830E7C280AA55
:100D4A0074F8CC6480CCC86480C8F582046043C35C
:100D5A00EB9FF5F0EA9E42F0E99D42F0E89C45F0EF
:100D6A0060305018E5825FFFE582F42B5582FB5014
:100D7A00210ABA001D09B90019088016E5825BFB31
:100D8A00E582F42F5582FF50090EBE00050DBD0005
:100D9A00010CC3EB9FF5F0EA9E42F0E99D42F0E8B0
:0D0DAA009C45F06007CC4820E701B3EC2227
:100DB700ED33EC33600A047003BD8004ECB2E7FC4A
:010DC7002209
:100DC80075F020800E75F010800575F0087D007EA6
:100DD800007F003392D530D503121322EC33401034
:100DE800EF33FFEE33FEED33FDEC33FCD5F0ED22AF
:0E0DF800E5F0247EA2D513CC92E7CDCEFF22EB
:100E0600EDD2E7CD33EC3392D524814006E4FFFEE4
:100E1600FDFC22FCE4CFCECDCC24E0501174FF8043
:100E2600EDC3CC13CCCD13CDCE13CECF13CF0470E0
:070E3600F030D5DE021322AB
:101A3100E54C2438F8E6054C227835300702783831
:101A4100E475F0011213F702116C2000EB7F2ED226
:101A5100008018EF540F2490D43440D4FF30040B8D
:101A6100EF24BFB41A0050032461FFE54D60021555
:101A71004D0550E5507002054F30070D7835E4757E
:101A8100F0011213F7EF0211B202354D7403D207C0
:101A91008003E4C207F54C8B358A368937E4F54D6E
:101AA100F54FF550E54D60077F20121A6C80F575F2
:101AB1004EFFC201C200C202C203C205C206C20871
:101AC100121A3AFF700D3007057F00121A7DAF50D0
:101AD100AE4F22B4255FC2D5C204121A3AFF24D0F8
:101AE100B40A00501A75F00A784D30D50508B6FFD2
:101AF1000106C6A426F620D5047002D20380D9249B
:101B0100CFB41A00EF5004C2E5D204021D6AD2011B
:101B110080C6D20080C0D20280BCD2D580BAD205A4
:101B210080B47F20121A6C2002077401B54D004069
:101B3100F1121A31FF121A6C021AA5D208D20680CC
:101B410095121A31FB121A31FA121A31F94A4B70F5
:101B51000679617A1E7BFF20022EE54D602A7E0008
:101B61008E8275830012118560060EEE654E70F04F
:101B7100C2D5EBC0E0EAC0E0E9C0E0EE121DCAD078
:101B8100E0F9D0E0FAD0E0FB12116CFF60AAEBC0E3
:101B9100E0EAC0E0E9C0E0121A6CD0E02401F9D01B
:101BA100E03400FAD0E0FBE54E0460DCD54ED9808C
:101BB10087D20280A2121DAD60F7E54E70010412BA
:101BC1000E87A94E600DE54E600914F54E121E54A4
:101BD100EF60F3EA30E702F404C3995077EAF425A1
:101BE1004E0430E701E404F54E800D121DAD60C1D5
:101BF100EA054E254E120E87EA784BF630E701E4EE
:101C0100254E04D54E0420050114121DCAE4C0E07E
:101C1100121E54784BE6601320E70714F6121A548B
:101C2100802204F6D0E014C0E07F00121A54E54E81
:101C31006007121A4B154E800B300503121A4BD058
:101C4100E0021AA5D0E00480C5121DAD60A0E54EEA
:101C510004120E87784BEAF6E54E20050260010476
:051C61002404121DCA5D
:101C660074FF04C0E0121E54121A54E54E200502F9
:101C76006003121A4BD0E0B54EE87F45121A5E7823
:101C86004BE67F2B30E7047F2DF404C0E0121A6C7C
:101C9600D0E075F00A84C0F0121A55D0E0121A5539
:101CA600021AA5791080027908C206C2088008D2F5
:101CB600D5790A8004790AC2D5E54E047002F54E3C
:101CC600E4FAFDFEFF121A31FC7B08200113121AFA
:101CD60031FD7B1030000A121A31FE121A31FF7BD9
:101CE60020EC3382D592D55013C3E43000069FFF13
:101CF600E49EFEE42001039DFDE49CFCE4CBF8C2D7
:101D060001EC700CCFCECDCCE824F8F870F3801738
:101D1600C3EF33FFEE33FEED33FDEC33FCEB33FB69
:101D2600994002FB0FD8E9EB300105F8D0E0C44832
:101D3600B201C0E00AEC4D4E4F78207B0070C2EA3B
:101D4600B54E0040BCC0E0121DCCD0F0D0E0200162
:101D560004C4C0E0C4B201C0F0121A55D0F0D5F0E8
:101D6600EB021AA51214171B42531CA9581B134C3D
:101D76001B0F421CAD4F1CB5441CB5491B28431C08
:101D8600BB551BEC461C4A451BB6471E81501B170C
:101D96002D1B1B2E1B3E2B1B1F231B3C201E6A2AA2
:101DA6001AD74800001B36E54EB4FF03754E0612DF
:101DB6001A31FC121A31FD121A31FE121A31FF784D
:101DC60044020EB6790AA2D5200314300509B910CB
:101DD600020404B9080104A2D52006025001042019
:101DE60002689202B54D005034C0E07F20300319DE
:101DF6007F30A20272067205500F121E23C202C263
:101E060006C205C2087F30800F300503E9C0E01224
:101E16001A6C300503D0E0F9D0E0B54DCC3005178B
:101E26007F30B9100C121A6C7F583004077F788007
:101E360003B90803121A6C3002057F2D021A6C7F53
:101E4600202008F87F2B2006F322920280CF7F0005
:101E5600B4070050052444F8E6FF22286E756C6C22
:101E66002900D201121A313001F8C201784D30D55D
:101E76000108F6021AD72D50434958121A31240385
:101E8600B405004001E4901E7C93121A5D743A1268
:0A1E96001A5DD203754D04021CA969
:10226600E54C30030104F82328243AF82278373065
:102276000302783AE475F0011213F702116C60EC70
:10228600C5507002154F14C550200304FF023809CB
:10229600783774FFF5F0021407FF023771E54D60D9
:1022A60006D54D037F002220030F1237A7EF6008E3
:1022B6000550E5507002054F2278371213EE1211C1
:1022C6006CFF60E97837E475F0011213F780DE12CF
:1022D60022ADEFC0E012229FD0E040F380A0D203EF
:1022E6008002C2038B378A388939E4F54EF54CF5FE
:1022F6004FF550754D00C202C200C201C20412223F
:1023060073FF7005AF4E7E0022B42530122273FF94
:1023160024D0B40A00500C75F00AC54DA4254DF51D
:102326004D80E924CFB41A00EF5002C2E5022581A0
:10233600D20180D8D20080D4D20480D0EF12229F5E
:1023460050081222D5EF600E80A9EFC0E01222AD30
:10235600D0E06F609EEF607412228480A71222ADD7
:10236600EF6069E54D7007054D80031222ADEF6001
:102376001420040E122266E475F0011213F7EF1210
:1023860011B2D54DE6200404054C054E80BA122242
:10239600A3EFC0E012229FD0E05004122284E4FF93
:1023A60020040E122266E475F0011213F7EF1211E3
:1023B600B2EF70DA200404054C054E808BE54D60C3
:1023C60002054D1222D51222A3EF70C6300304E493
:1023D600122284E54E600302230A7EFF7FFF22E578
:1023E6004D6002054D1222D5D206D2051222A3EF68
:1023F60030060260D7C0E0122284D0E0AC51AD5264
:10240600AE53AF54122E638C518D528E538F54504F
:10241600071222ADC20580D4200410200502054E05
:082426001222661213EE054CB0
:10242E001213770222F9D0E0809A7900800A79108F
:10243E00800679088002790AD205E54D6002054DC5
:10244E00E9C0E01222D5EF60DD1222ADBF2D04D21D
:10245E00028003BF2B091222D5EF60CA1222A3D02D
:10246E00E0B40A028033B40802802EBF3027700217
:10247E007408C205C0E01222A3D0E0BF7802800328
:10248E00BF5816054DD54D028007D54D04D2058097
:10249E000B741080197002740ABF000AEFF8E4FC86
:1024AE00FDFEFF022534C0E0EF122284D0E0F9E4F5
:1024BE00FCFDFEFFE9C0E0ECC0E0EDC0E0EEC0E0E8
:1024CE00EFC0E01222A3EFF8D0E0FFD0E0FED0E0A4
:1024DE00FDD0E0FCD0F0E8604DB461004007B47B65
:1024EE00005002C2E524D0503DFA24F6500724F9DC
:1024FE005034240AFAEAB5F000502BCFA9F0A42FDD
:10250E00FF92D5E9C5F0CEA4A2D53EFE92D5E9C57F
:10251E00F0CDA4A2D53DFD92D5E9C5F0CCA4A2D5AF
:10252E003CFCC205808EE8C0E020042A2005080588
:10253E004E3002031213221222661213EE054C20A5
:10254E00000B20010DEE8FF01211E68009121377A9
:10255E008004EF1211B2D0E01222840222F920047C
:10256E00101222661213EE054CE54F8550F0121133
:10257E00E680E812141723C353243C58233A4C2305
:10258E00364223124824404F2444442363432438C4
:10259E004924445523E54623E54523E547233E2AB2
:0725AE00256C4E00002342E2
:0D37C700ED33EC3360065004EC6480FC220E
:102F3600020E7222EDA2E7D2E7F9EC3340F260F31B
:102F4600B4FF08ED547F70E8020E7CF82481C2E0DD
:102F5600C0E0F40428FAC313FCED92E7FD8C448D1F
:102F6600458E468F47EEA2E7E9BA7F02C3133400C7
:102F76009400FA75F091A4E5F013F494FE8AF0A497
:102F860033E5F033248CD313FDE492E7FE7F007C17
:102F96003F758302ECC0E0F8EDC0E0F9EEC0E0FA60
:102FA600EFC0E0FBAC44AD45AE46AF47120CADD02A
:102FB600E0FBD0E0FAD0E0F9D0E0F8120AB3ED6415
:102FC60080FD30E7011CD583CBED33CC33F8D0E060
:0A2FD600A2E71328C313CC13FD2259
:10316C008F478E468D458C44AB4BAA4AA949A8483B
:10317C00120CAD122A188F478E468D458C44E548AB
:10318C0030E747ECC0E0EDC0E0EEC0E0EFC0E0E4BB
:10319C00FFFEFDFCAB47AA46A945A844120D4A7B8D
:1031AC00DB600250087A0F7949784080067A0F79F3
:1031BC004978C0D0E0FFD0E0FED0E0FDD0E0FC12BA
:1031CC000AB38F478E468D458C44AF47AE46AD450E
:0331DC00AC4422DE
:102742003A70FA83BCAAE9E43E81E0F8BF9DE9E66B
:102752003F80000039283C1ABB9969663DA335E3E6
:10276200BF255DE73FC90FDB418DDBCCC44936EEA7
:1027720045C9913FC5B0F83D3F800000C317F5340D
:10278200452FFA73C60AFDDD12283104A2E1920038
:102792001420E0159027427404120FB980261228E3
:1027A2003130E102B20020E0EB8C448D458E468F41
:1027B200479027567404120FB9A844A945AA46ABFC
:1027C20047120BA4ED4C6007300004EC6480FC223D
:1027D200122831C0E08C448D458E468F4790277A6F
:1027E2007403120FB9A844A945AA46AB47120BA419
:1027F200ECC544FCEDC545FDEEC546FEEFC547FF01
:1028020090276A7403120FB9D082A844A945AA4638
:10281200AB47E58230E007120CADB20080A6EFCBE9
:10282200FFEECAFEEDC9FDECC8FC120CAD8095EDC1
:1028320033EC547FCC33920024605007D0E0D0E0D8
:10284200020E727B837AF97922783E120BA4EDF99B
:1028520033ECF83324815011EFFBEEFA120E06121C
:102862000DC8ECB2E7FC120AB3ED33EC33602F244F
:1028720003F8C313FCED92E7FDE82481E4501FEC5A
:10288200F8EDF9EEFAEFFB120E06EF04C2E0FCF5EA
:1028920082120DD2ECB2E7FC120AB3E58203FAED22
:0E28A20033EC3360071413FCED92E7FDEA22DD
:100E3D00E9D2E7C933E833F892D5EDD2E7CD33ECFB
:070E4D0033FC5002B2D52274
:100E5400EC30E7100FBF000C0EBE00080DBD0004FF
:100E64000BEB6014A2D5EB13FCED92E7FD2274FFAB
:100E7400FCFDFEFF22E480F8A2D574FF13FC7D8004
:030E8400E480EF18
:100E8700F920E72824F950037907E4F42402FB1832
:100E9700DBFDE624FB5014E9600DE4F618E604F6E2
:0F0EA700B40A08E4F6D9F57401F60A22C2D5227E
:100EB600ED33EC3392D5FA602AB4FF33EDC2E77B0B
:100EC600FF60067A0E79DBE4227A0E79E420D504F7
:100ED6007A0E79DF224E614E002B494E46002D498F
:100EE6004E4600E47A08F608DAFC7B00740722E82E
:100EF600C0E0ECC0E0EDC0E0EEC0E0EFC0E0EA75B7
:100F0600F010A4CAABF075F04DA42BFBE435F0FC51
:100F1600EA2410FAEB34C5FBEC34D9FCEDC2E7FF4A
:100F260075F056A4F42411C5F0F434C58FF0A42A44
:100F3600E5F03BE43CF620E714121036D0E0FFD093
:100F4600E0FED0E0FDD0E0FC120CAD8014F40412FB
:100F56001036D0E0FFD0E0FED0E0FDD0E0FC120B72
:100F6600A4D0E0F8E6FAEDD2E7CD33EC332482FBE9
:100F7600E4C3CF33CFCE33CECD33CD33DBF37B07D4
:100F860075F00A846004F6081B0AE5F0F6088FF08F
:100F9600740AA4FFACF08EF0740AA42CFEACF050D8
:100FA600010C8DF0740AA42CFDE435F0F608DBDEA6
:030FB6007407229B
:102E5000C207C208C209C20AF9E4F555F556FCFDDD
:102E6000FEFFE91006EA20090CB42D04D209D32292
:102E7000B42B02D32224D0504794095041240A3065
:102E80000A15F88556F0740AA42872E74051C5F077
:102E9000704D85F056D322D208C0E0E4FBFA7920C9
:102EA0007841120BA4ECF8EDF9EEFAEFFBD0E0FC60
:102EB000E4120DD2120AB33007B41555D322240AF6
:102EC000200A20B4FE0720071AD207D32224EB6081
:102ED0000424E0700EA2099207D20AC209D322C3C9
:102EE000020E72E4300A0BE556300902F404A20720
:102EF00092093008EA255520D2E5A2E7920A50024D
:102F0000F404B4260050D8CCC0E0EDC0E0EEC0E040
:102F1000EFC0E0EC121036D0E0FFD0E0FED0E0FDD4
:102F2000D0E0FC200A05120BA48003120CAD30097E
:062F300003120DB7C322DD
:100FB900C0E0EFFBEEFAEDF9ECF8120BA4D0E0F586
:100FC900F0EFFBEEFAEDF9ECF8121391A3A3A3A34A
:100FD900E8C0E0E9C0E0EAC0E0EBC0E0C0F0120B15
:100FE900A41213A1A3A3A3A3120AB3D0F0D0E0FBC8
:0D0FF900D0E0FAD0E0F9D0E0F8D5F0D42235
:1029F800BE1249253E4CCCCDBEAAAAAB3F800000F2
:102A08003E7ADBB03EED63383F24BC7D3F490FDBA7
:102A1800ED33ECC2E7CC339200B4FF13ED547F6082
:102A280003020E727FDB7E0F7DC97C3F022B13C22F
:102A380001C3947F401E7007EDD2E794904015EFD4
:102A4800FBEEFAEDF9ECF87F007E007D807C3F120A
:102A58000CADD201ED33EC33248430E705E4C0E05B
:102A6800806D04FAEDD2E754F0C333DAFD5407342D
:102A7800002323C0E0CCC0E0F8EDC0E0F9EEC0E0F0
:102A8800FAEFC0E0FBE4120DD2EC24FEFC8C4C8D76
:102A98004D8E4E8F4F120BA47B007A007980783FC1
:102AA800120AB3ECC54CB2E7FCEDC54DFDEEC54EC0
:102AB800FEEFC54FFFD0E0FBD0E0FAD0E0F9D0E060
:102AC800F8120AB3A84CA94DAA4EAB4F120CAD8C04
:102AD8004C8D4D8E4E8F4F9029F87403120FB9A864
:102AE8004CA94DAA4EAB4F120BA4D0E0600F2404A2
:102AF800F582E4342AF5831213A1120AB330010BCC
:102B08007BDB7A0F79C978BF120AB3ED33EC3360F7
:082B180006ECA20092E7FC228A
:101006003F8000004120000042C80000447A0000F2
:10101600461C400047C35000497424004B18968074
:101026004CBEBC205A0E1BCA6753C21C749DC5AE6B
:10103600FB60065407601C2323121064EB543860CF
:101046000912105012105F120BA4ECF8EDF9EEFA2B
:10105600EFCB22EB12105F80F1543803241C901062
:1010660006FE93FC0EEE93FD0EEE930ECE93FF223C
:102FEC00022D60E493A3F8E493A34003F68001F26E
:102FFC0008DFF48029E493A3F85407240CC8C333E6
:10300C00C4540F4420C8834004F456800146F6DFB4
:10301C00E4800B0102040810204080903804E47E08
:10302C00019360BCA3FF543F30E509541FFEE493A9
:10303C00A360010ECF54C025E060A840B8E493A370
:10304C00FAE493A3F8E493A3C8C582C8CAC583CA9B
:10305C00F0A3C8C582C8CAC583CADFE9DEE780BE53
:0138080000BF
:10107600E709F608DFFA8046E709F208DFFA803E5C
:1010860088828C83E709F0A3DFFA8032E309F60849
:10109600DFFA8078E309F208DFFA807088828C83B1
:1010A600E309F0A3DFFA806489828A83E0A3F60865
:1010B600DFFA805889828A83E0A3F208DFFA804C3F
:1010C60080D280FA80C680D4806980F28033801016
:1010D60080A680EA809A80A880DA80E280CA80337F
:1010E60089828A83ECFAE493A3C8C582C8CCC583F7
:1010F600CCF0A3C8C582C8CCC583CCDFE9DEE780C7
:101106000D89828A83E493A3F608DFF9ECFAA9F045
:10111600EDFB2289828A83ECFAE0A3C8C582C8CC9B
:10112600C583CCF0A3C8C582C8CCC583CCDFEADEB4
:10113600E880DB89828A83E493A3F208DFF980CC16
:1011460088F0EF60010E4E60C388F0ED2402B4040F
:101156000050B9F582EB2402B4040050AF232345B6
:0611660082239010C67305
:10116C00BB010689828A83E0225002E722BBFE0281
:09117C00E32289828A83E49322B4
:10118500BB010CE58229F582E5833AF583E022501F
:1011950006E92582F8E622BBFE06E92582F8E22269
:0D11A500E58229F582E5833AF583E4932283
:1011B200BB010689828A83F0225002F722BBFE011C
:0211C200F32216
:1011C400F8BB010DE58229F582E5833AF583E8F061
:1011D400225006E92582C8F622BBFE05E92582C80D
:0211E400F222F5
:1011E600BB010A89828A83F0E5F0A3F0225006F754
:0F11F60009A7F01922BBFE06F3E5F009F3192251
:10120500E88FF0A4CC8BF0A42CFCE98EF0A42CFC88
:101215008AF0EDA42CFCEA8EF0A4CDA8F08BF0A406
:101225002DCC3825F0FDE98FF0A42CCD35F0FCEB65
:101235008EF0A4FEA9F0EB8FF0A4CFC5F02ECD392A
:0F124500FEE43CFCEAA42DCE35F0FDE43CFC2297
:1012540075F008758200EF2FFFEE33FECD33CDCC51
:1012640033CCC58233C5829BED9AEC99E5829840D4
:101274000CF582EE9BFEED9AFDEC99FC0FD5F0D6B1
:10128400E4CEFBE4CDFAE4CCF9A88222B800C1B9DB
:101294000059BA002DEC8BF084CFCECDFCE5F0CB19
:1012A400F97818EF2FFFEE33FEED33FDEC33FCEB52
:1012B40033FB10D703994004EB99FB0FD8E5E4F90D
:1012C400FA227818EF2FFFEE33FEED33FDEC33FCFA
:1012D400C933C910D7059BE99A4007EC9BFCE99AEE
:1012E400F90FD8E0E4C9FAE4CCFB2275F010EF2F33
:1012F400FFEE33FEED33FDCC33CCC833C810D70733
:101304009BEC9AE899400AED9BFDEC9AFCE899F86D
:0E1314000FD5F0DAE4CDFBE4CCFAE4C8F92200
:0E132200C3E49FFFE49EFEE49DFDE49CFC22DC
:10133000EB9FF5F0EA9E42F0E99D42F0EC6480C834
:0613400064809845F022D4
:10134600EB9FF5F0EA9E42F0E99D42F0E89C45F0FD
:011356002274
:10135700BB010789828A830214495005E9F8021400
:101367003DBBFE05E9F802145589828A8302139171
:10137700BB010789828A830213B15005E9F8021479
:0A13870061BBFE05E9F802146D22B7
:10139100E493FC740193FD740293FE740393FF22A2
:1013A100E493F8740193F9740293FA740393FB22A2
:0C13B100ECF0A3EDF0A3EEF0A3EFF022AF
:1013BD00A8828583F0D083D0821213D41213D41255
:1013CD0013D41213D4E473E493A3C583C5F0C5837A
:1013DD00C8C582C8F0A3C583C5F0C583C8C582C87A
:0113ED0022DD
:0913EE00E6FB08E6FA08E6F92224
:1013F700FAE6FB0808E6F925F0F618E6CA3AF622F7
:10140700FAE6FB0808E625F0F9F618E63AFAF622B6
:10141700D083D082F8E4937012740193700DA3A364
:1014270093F8740193F5828883E473740293686078
:06143700EFA3A3A380DF78
:10354D00EFB40A07740D123558740A309811A89902
:10355D00B8130CC2983098FDA899C298B811F630DE
:07356D0099FDC299F59922B6
:1037A70010180B1237DEBF0D027F0A02354DAF0F1F
:0137B70022EF
:053809008F0FD2182210
:10377100EFC394094005EF940E4003BF2003D380AB
:0337810001C3225F
:103298008B2E8A2F89308B348A358936AB2E0530B0
:1032A800E530AA2F7002052F14F912116C70ED7415
:1032B800FF2530F53074FF352FF52FAB310533E599
:1032C80033AA327002053214F912116CFFAB2E05C5
:1032D80030E530AA2F7002052F14F9EF1211B270E1
:0832E800DAAB34AA35A9362245
:10000E00E4FFFE12116C600C0FEF70010E09E97027
:05001E00F20A80EF2250
:0C143D00E6FC08E6FD08E6FE08E6FF22DB
:0C144900E0FCA3E0FDA3E0FEA3E0FF2216
:0C145500E2FC08E2FD08E2FE08E2FF22D3
:0C146100ECF608EDF608EEF608EFF622B7
:0C146D00ECF208EDF208EEF208EFF222BB
:0A37DE003098FDAF99C2987E0022DA
:00000001FF
